:100000000C9434000C944F000C944F000C944F004F
:100010000C944F000C944F000C944F000C944F0024
:100020000C944F000C944F000C944F000C944F0014
:100030000C944F000C944F000C944F000C944F0004
:100040000C944F000C944F000C944F000C944F00F4
:100050000C944F000C944F000C944F000C944F00E4
:100060000C944F000C944F0011241FBECFEFD4E02E
:10007000DEBFCDBF11E0A0E0B1E0E4EDF0E002C0F2
:1000800005900D92A030B107D9F711E0A0E0B1E0E2
:1000900001C01D92A030B107E1F70C945E000C94F2
:1000A00000009C01E0E8F7E005C0CF010197F1F7FF
:1000B0002150304021153105C1F708953D9A4598EA
:1000C00082E390E00E945100459A82E390E00E9412
:0400D0005100F5CF17
:00000001FF
